:1000000012C0189518951895189518951895189563
:100010001895189518951895189518951895189578
:100020001895189518958FE58DBFC0E4E8E34E2E1E
:1000300084E08EBFD4E0F4E05F2EEEEFF3E0A0E6C4
:10004000B0E088278D933197E9F7DDD066248CE006
:1000500022D1A098A89A8F98979A80E08093600008
:1000600080E08093610081E080936200B5D0B0D0E1
:10007000E2EEF3E0A7D0A3E3B0E08C9180FBA3E62F
:10008000B0E08C9187F98C930027A3E6B0E08C91C7
:1000900087FB0EF401E040E0041709F001C075D0C1
:1000A0000027A0E3B0E08C9187FB0EF401E040E074
:1000B000041709F001C054D08FEB11E09CD0E8EE9A
:1000C000F3E080D0A0E2B4E0E2E6F0E040D172D00C
:1000D000EAEEF3E077D0A0E2B4E0E1E6F0E037D179
:1000E00069D0EAEEF3E06ED0A0E2B4E0E0E6F0E042
:1000F0002ED160D083EE93E0FAD0A0E6B0E08C91F0
:100100008F5F8C93009160000B3310F009F001C0F9
:1001100024C080E080936000A1E6B0E08C918F5F06
:100120008C9380E1B8D0E8EEF3E04CD00091610010
:100130000B3310F009F001C010C0A2E6B0E08C91C2
:100140008F5F8C9380E080936100009162000C309F
:1001500010F009F001C001C080CF8DCFF894FFCF1F
:10016000A1E6B0E08C918F5F8C93009161000B331E
:1001700010F009F001C008C02FD02AD0E2EEF3E061
:1001800021D080E0809361000895A2E6B0E08C91D8
:100190008F5F8C93009162000C3010F009F001C069
:1001A00008C081E08093620017D012D0E2EEF3E045
:1001B00009D00895A0E2B4E08D91882311F065D0B4
:1001C000FBCF0895A3D0802D11F05FD0FBCF089511
:1001D00082E061D015D011C081E05DD011D080E8FF
:1001E0005AC08FE7213039F08FEB223021F08FE8B1
:1001F000233009F08FEC810F4EC080E84CD0089579
:1002000083E0992774C08AEF90E071D0A49AA39AF2
:10021000A29AA19A8A9A8B9A939885E090E067D0E7
:100220009298AC98AB98AA9AA99A929AEF93FF9356
:10023000E4ECF0E050D0FF91EF91929855D0929A73
:10024000EF93FF93E4ECF0E046D0FF91EF919298AA
:100250004BD0929AEF93FF93E4ECF0E03CD0FF9107
:10026000EF91929841D0A998929AEF93FF93E4EC82
:10027000F0E031D0FF91EF91929836D088E20BD028
:100280008EE009D086E007D00895939A829505D034
:1002900004D02AD008959398F9CF859510F4A99A9F
:1002A00001C0A998859510F4AA9A01C0AA988595CD
:1002B00010F4AB9A01C0AB98859510F4AC9A01C0CC
:1002C000AC98929AEF93FF93E4ECF0E004D0FF91A6
:1002D000EF91929808953197F1F70895689462F834
:1002E0000895E89462F8089581E090E000C0EF93EB
:1002F000FF93EE27E82BE92B31F0E0EDF7E03197A3
:10030000F1F70197D1F7FF91EF910895C8953196D4
:1003100000200895000F111F221F331F089500951C
:100320001095209530950F5F1F4F2F4F3F4F089529
:10033000019110810EC001911191219130810BC06A
:100340000191108117FF05C03FEF2FEF04C000811E
:1003500011272227332737FF03C0E1DF8DE28D937A
:10036000CF93DF93CF92DF92EF92AA24BB24CC24C9
:10037000DD24EE2440E2CAE0DD2755E093E38881E6
:10038000890F87FD9F7083FD907F891B89935A9504
:10039000A9F7C0DFAA1CBB1CCC1CDD1CEE1C4A95B7
:1003A00051F7E894EFE0FF2782910ED0EB30E0F7B1
:1003B0001EF068948A2D0CD088278D93EF90DF90E3
:1003C000CF90DF91CF910895982F829501D0892FFA
:1003D0008F70805D26F0803309F4089568948D93C2
:0C03E000089574696D653A0000003A0051
:00000001FF
